:1000000014C02EC02DC02CC02BC02AC029C028C0AF
:1000100027C0B3C025C024C023C022C021C020C037
:100020001FC01EC01DC00D0A000011241FBECFE559
:10003000D4E0DEBFCDBF10E0A0E6B0E0E2E5F6E040
:1000400002C005900D92A236B107D9F710E0A2E6E2
:10005000B0E001C01D92A139B107E1F751D0F7C25C
:10006000CFCF9B9902C081E008959A9902C082E0A7
:100070000895999902C083E00895989902C084E098
:100080000895B59902C085E00895B49B02C080E050
:10009000089586E0089597989698959894989398DF
:1000A0009298833091F0843028F4813051F082307E
:1000B00099F409C0853069F0853048F0863061F4E4
:1000C0000AC0979A0895969A0895959A0895949AD1
:1000D0000895939A0895929A089580E090E07ED2D0
:1000E000853521F481E090E079D2089580E090E0B8
:1000F00065E57CD281E090E061E078D281E008950E
:100100000F931F9380E388BB8FE085BB80E284BBA5
:100110008EEF81BB81E089BF83BF78949B9913C028
:1001200011E0812F04D1812FB6DF04C083B3829503
:100130008170B8D014D18130C9F311D1823019F057
:100140001F5F173071F7C9DFA6DFAD9A00E089DFC6
:10015000182F882311F4F8D0182F011749F0112314
:1001600039F081E090E0612F41D2812F94DF012F9F
:1001700083B38295817096D0EACF1F920F920FB60B
:100180000F9211242F933F934F935F936F937F931D
:100190008F939F93AF93BF93EF93FF9353D1FF91AF
:1001A000EF91BF91AF919F918F917F916F915F91EF
:1001B0004F913F912F910F900FBE0F901F90189568
:1001C0008AB188618AB980B5866880BD8CE089B9BA
:1001D00010BC579A08955D9BFECF8CB90895FC0121
:1001E00004C05D9BFECF8CB9319680818823C9F70E
:1001F000089503C05D9BFECF2CB9FC0101962491AC
:100200002223C1F7089586E290E0F3DF0895DF939B
:10021000CF93CDB7DEB761970FB6F894DEBF0FBEB0
:10022000CDBFBE016F5F7F4F4AE050E0B8D1D7DF4E
:1002300061960FB6F894DEBF0FBECDBFCF91DF91B0
:100240000895982F80916200883058F5E0916200FF
:10025000F0E0E757FF4F8081880F80838091640032
:100260008F5F8093640080916400883039F410922D
:100270006400809162008F5F8093620060916500EE
:10028000892F7AD1833040F0E0916200F0E0E757A7
:10029000FF4F80818F5F8083809163008F5F8093A9
:1002A00063000895882361F590916C009130F1F519
:1002B000AD9810926C0080916B00882319F4909394
:1002C0006B0019C080916B00813061F480916800EF
:1002D00090916900909367008093660082E080931C
:1002E0006B0009C080916B00823001F5809168003D
:1002F00090916900A6DF109269001092680008953D
:1003000080916C00882391F481E080936C0080914F
:100310006B00823059F480916200882339F4809117
:10032000680090916900825080936500089587303D
:1003300020F480936D0081E001C082E08093600032
:10034000089510926D00089580916A00882331F01D
:1003500080917000882311F01092700008958091B0
:1003600060000895EF92FF920F931F93CF93DF9356
:1003700000E08CE0E82EF12CC0E0D0E0FE01E75771
:10038000FF4F1081C7018C0F9D1F28D1181729F42A
:100390002196C830D10591F708C00F5F8AE090E040
:1003A000E80EF91E063041F703C00F5F009370009E
:1003B000DF91CF911F910F91FF90EF9008950F93D0
:1003C0001F93CF93DF9300916D008AE0089F800117
:1003D000112460916500C80109D10F5F1F4F609122
:1003E0006300C80103D1C0E0D0E00F5F1F4FFE01E2
:1003F000E757FF4F6081C801F9D02196C830D10579
:10040000A1F7DF91CF911F910F91089521E730E07F
:10041000C90160E070E048E150E0BAD0089529E8F1
:1004200030E0C90160E070E048E050E0B1D01092E7
:100430006A001092620010926400109263001092A1
:1004400070000895CF93DF938091680090916900C8
:100450008A3F910558F080916B008130A9F480911A
:100460006800909169008E55914070F480916A0007
:100470008111D5DF80916800909169000196909379
:1004800069008093680075C080916B00882309F42F
:1004900070C0AD9A10926B0081E080936A008091E9
:1004A0006D00882309F464C020E030E0E0916E0024
:1004B000F0E0D901A757BF4F8C9143E0EE0FFF1F2B
:1004C0004A95E1F7E20FF31FEF58FF4F80832F5F4C
:1004D0003F4F2830310551F780916E008F5F809338
:1004E0006E0080916E00833011F410926E0041E036
:1004F00050E018C0C1E7D0E0F901EC0FFD1F90817A
:10050000FB01E20FF31FEC0FFD1F80819817C9F468
:100510002F5F3F4F2830310569F74F5F5F4F433002
:10052000510549F020E030E0BA0193E0660F771FF3
:100530009A95E1F7DFCF43DF1092600010926D00D3
:100540000EC080916F008F5F80936F0080916F006D
:100550008A3079F410926D0082E0809360001092EE
:100560006F00CE0160E070E048E150E011D001C0C2
:10057000F9DEDF91CF910895991B79E004C0991FAE
:10058000961708F0961B881F7A95C9F780950895ED
:10059000DC0101C06D9341505040E0F70895FB012C
:1005A0009F01E8944230BCF04532ACF44A3029F463
:1005B00097FB1EF4909581959F4F642F772733D03A
:1005C000805D8A330CF0895D8193CB010097A9F798
:1005D00016F45DE251931082C90115C0E199FECF76
:1005E0009FBB8EBBE09A99278DB30895262FE19982
:1005F000FECF9FBB8EBB2DBB0FB6F894E29AE19A5B
:100600000FBE01960895DC01FC01672F71917723DD
:10061000E1F7329704C07C916D9370836291AE17BD
:10062000BF07C8F30895AA1BBB1B51E107C0AA1F4F
:10063000BB1FA617B70710F0A61BB70B881F991F83
:100640005A95A9F780959095BC01CD010895F8942D
:02065000FFCFDA
:020652000100A5
:00000001FF
